:0CFF000041003F00000000000000000075
:03000000020AD21F
:100AD200208003021F0078FFE4F6D8FD7581AB0287
:020AE2000B1FE8
:10159F00C2AF53F17F8FF3E5F130E7FBAFF2D2AF7C
:0115AF002219
:1015B000C2AF53F17F8DF28FF3E5F130E7FBD2AF8D
:0115C0002208
:100F120020204D555445204F4E2020200080800037
:100F22007040302010100818041C00FBF7F3EFEBA0
:100F3200E7E3DFDBD7D3CFCBC7C3BFBBB7B3AFAB1F
:100F4200A7A39F9B97938F8B87837F7B77736F6B0F
:100F520067635F5B57534F4B47433F3B37332F2BFF
:0A0F620027231F1B17130F0B0703B3
:100DF500079C0A0A0A0A0A0A0A01A306019900C100
:050E05001D02200000A9
:041154008E298F2A27
:10115800E4F52B7F017E0012149BE52A30E004D2CF
:10116800868002C286C2857F017E0012149BD285CA
:10117800E529C313F529E52A13F52A052BE52BC321
:04118800941040CFB0
:01118C002240
:10157900AF21AE20121154C2847F017E0012149B48
:03158900D28422E7
:041098008E298F2AE4
:10109C00E4F52BE52A30E004D2868002C286D285A4
:1010AC007F057E0012149BC2857F0A7E0012149B62
:1010BC00D2857F057E0012149BE529C313F529E523
:0D10CC002A13F52A052BE52BC3940D40C611
:0110D90022F4
:02145D00AC07DA
:10145F00ECFFEFFEEDFF6307FF6306FFD283121071
:0C146F0098C2837F057E0012149BD2837C
:01147B00224E
:10130C00301106C200C208801130920AC200C20815
:10131C00D201D2098008D200D208C201C209789B3E
:10132C00E66004C200C201789AE66004C208C209F1
:03133C000215791E
:0B160E00C201C200789B760102157932
:0B161900C209C208789A760102157918
:100B6400E4F527F5288F278F2878A3E6FEC394069B
:100B74005018C374069EF527EFC394385007E52731
:100B84002FF527802075273E801BEED39406401551
:100B9400EE24FAF528EFC394385007E5282FF528FA
:100BA400800375283EE527700512160E8012E4783E
:100BB4009BF6E527900F2D93F527FD7F1812145D02
:100BC400E52870051216198012E4789AF6E5289043
:100BD4000F2D93F528FD7F1C12145DA21D921102A6
:020BE400130CF0
:10118D008F27D21112130C7F647E0012149B5321F2
:10119D0003532003E52725E0241FF582E4340FF5E2
:1011AD0083E493422074019342211215797FC87E06
:0911BD000012149BC21102130C74
:100E0A00C11A021A0000011900011D00021E000089
:030E1A00011800BC
:100F6C00E51A5407FEE51B54C07003EE640170349F
:100F7C00E51BB51F1EE51AB51E19E51C640D6006B0
:100F8C00E51C642C702B0518E518B40324D219E465
:100F9C00F51822E4F518E51B543FF51CD219851AF7
:100FAC001E851B1FE4F51D751901F51A751B01D261
:010FBC001A1A
:010FBD002211
:03000B000210DA06
:1010DA00C0E0C0D075D000C006C28C758A00758C7D
:1010EA00D0E519641A6005E519B4190EE51B25E067
:1010FA00F51BE51A33F51A120F6C751D00751901E7
:0F110A00751A00751B01D21AD006D0D0D0E03272
:10073200C28CAF8CEFFEAD8A7C00E42DFFEC3EABA9
:1007420007FAE4F58A758CD0D28CD3EB94E0EA9464
:10075200D9400EEB94E0EA94DF50067A007B0280E7
:100762002FD3EB94A0EA94E0400EEB94A0EA94E637
:1007720050067A007B038018D3EB9400EA94E84099
:100782000BEA94EE50067A007B0480047A007B0127
:10079200E51B13921AE51D7010751D01751901F5FF
:1007A2001A751B01D21A020833EA701CEB24FD6091
:1007B2000D14600E2402701005190519800A7403C5
:1007C200800274042519F519E51B25E0F51BE51ACD
:1007D20033F51AE51930E020EA7056EB24FD600C7F
:1007E20014600E2402704A301A478032301A248074
:1007F20032301A02801D802BAE02AF03EA7032EF54
:1008020024FD600C14600924027026301A23800E25
:10081200301A10E51B25E0F51BE51A33F51A431BC8
:1008220001800E431B01E51B25E0F51BE51A33F59C
:100832001AE519B41B03120F6CE519D3941B40037C
:03084200E4F51DBD
:010845002290
:0300130002158C47
:10158C00C0E0C0D075D008C2AF120732D2AFD0D0F5
:03159C00D0E0326A
:101508002D4F46462D00204341525920415544490C
:081518004F200056312D320076
:0E0E1D00014100C11E04A580888B8F01A40234
:1012D80030100F7899E6249CF8E6C3943E500D062A
:1012E800800A7899E6249CF8E6600116C21D789970
:1012F800E6249CF8E6FF120B647899E6249CF8E64D
:04130800FF02139E2F
:101119008F2612118D75F003E526A424BDF582E50D
:10112900F0340AF583E493FB740193FA740293F99A
:101139007D097F01120EB7749C2526F8E6FF120B74
:0B11490064749C2526F8E6FF02139E4C
:1011FE0030100B78A3E6C3940C501206800F78A320
:10120E00E6FFD3940C5006EF94004001167899E651
:10121E00249CF8E6FF120B6412160278A3E6FF1266
:07122E0008467FC80215F21B
:10061700D21112130C78A97600087664D378AAE66B
:0B062700940018E6940050F4301E59B7
:100632001215377BFF7A1579087D097F05120EB7EF
:10064200121053E4F52678A97600087614D378AA16
:10065200E6940018E6940050F4B2930526E526B419
:1006620009E4C21EC28212126CC28178A976000805
:100672007632D378AAE6940018E6940050F4121564
:0606820037121053D2876D
:10068800020719D21EC287D281D29378A9760008B0
:100698007664D378AAE6940018E6940050F478A417
:1006A800E624A5F8E6FF1215E27BFF7A15790E7DA0
:1006B8000D7F01120EB7121053D28278A976030863
:1006C8007620D378AAE6940018E6940050F4789936
:1006D800E6FF12118D7899E675F003A424BDF58222
:1006E800E5F0340AF583E493FB740193FA740293FA
:1006F800F97D097F01120EB77899E6249CF8E6FF88
:10070800120B647899E6249CF8E6FF12139E1210E7
:100718005378A97600087614D378AAE6940018E6E8
:0A072800940050F4C2197543FF223B
:1012A3001216027BFF7A15791B7D087F05120EB794
:1012B3007FC81215F2E4FF7E07789C740AF608DEF5
:1012C300FC789CE6FF120B6478A37606E47899F623
:0412D30078A4760283
:0112D70022F4
:1004F0008F2512001E1215C1201E1AE52524BA6090
:100500000E24ED600D14600A243660030206160204
:1005100005D702060CE5251209E6056D0D059F12AB
:1005200005A61305AE1405B61505BE1605C61905B4
:10053000CE1A05721D05D72405E32905692C058E01
:100540003105823305DE3805DA3D05D74705765497
:1005500005FD5505F75605F15705EB58060A5906EE
:100560000C5A0613DD00000616D2108002C21002DB
:1005700012D8B21D8002C21DA21D921112130C02CC
:1005800014B7789906E675F00784A6F0800E78997E
:10059000E66003168004789976067899E68004E48C
:1005A0007899F6FF802E789976017F0180267899D8
:1005B00076027F02801E789976037F0380167899F1
:1005C00076047F04800E789976057F0580067899F9
:1005D00076067F06021119020617C2108002D21099
:1005E0000211FE78A4E6045403801578A4760380F3
:1005F0001078A47602800A78A476018004E478A4B6
:10060000F6E624A5F8E6FF0215E28000A21D92118D
:0706100002130C1212A322D9
:1013CB00E4FEEE25E024D2F582E43415F583E493B4
:1013DB00B50710EE25E024D3F582E43415F583E44C
:0913EB0093FF220EBE08DB7FFF18
:0113F40022D6
:100D9000E4FF12147CEF600A7542011213CB8F43FB
:100DA000802930190AC219E4F542851C43801CE5EC
:100DB00043B4FF1712133FBF010375432CBF020357
:100DC00075430DEF70051211C68F4320801978A965
:100DD0007600087601D378AAE6940018E6940050CD
:100DE000F4208003754324E543F46008AF43120404
:040DF000F07543FF58
:010DF40022DC
:1015D200011210130214201504164019081A09DD0D
:070E2B00014700C11BC19C3F
:10147C00E4C2A47F421214D37F017E0012149B128B
:0E148C001520D2A4E547B507037F00228F4745
:01149A00222F
:10133F00A2A0301B01B340037F00227F327E001238
:10134F00149BA2A0301B01B340037F0022A2A092E6
:0F135F001B301B0930A1037F01227F02227F0078
:01136E00225C
:1011C600A292301C01B3502D78A97600087601D37F
:1011D60078AAE6940018E6940050F4A292301C0116
:1011E600B35006A292921C80037FFF22301C037F1D
:0711F6005A227F59227FFFFE
:0111FD0022CF
:10149B00EF7802C333CE33CED8F9FFD3EF9400EEFF
:0C14AB0094004007EF1F70F31E80F02239
:1014EE00E4F58475856A7580FF75910C75920875A3
:0A14FE0090FFF5A4F5A575A0FF22EC
:05000E00D28AD2AA22F3
:03001600D2AF2244
:10123500E4FF12159F7899A6077F0112159F78A3E1
:10124500A6077F0912159F78A4A607E4F524E524CF
:101255002402FF12159F749C2524F8A6070524E592
:0612650024C3940740E8D9
:01126B002260
:10126C007899E6FDE4FF1215B078A3E6FD7F011234
:10127C0015B078A4E6FD7F091215B0E4F527E52733
:10128C002402FF749C2527F8E6FD1215B00527E50E
:06129C0027C3940740E89F
:0112A2002229
:100E57007F0A12159FEF64A560247DA57F0A1215EE
:100E6700B07F07789C740AF608DFFC7F0778A376C3
:100E770006E47899F678A4760212126C802B121287
:100E87003578A3E6D3940C4002760678A4E6D3948B
:100E970003400276027899E6D394074002E4F67895
:0F0EA7009CE6D3943E4002760AD287C293C28261
:010EB6002219
:040E320002A9000011
:07163900758911E4F58F2211
:0A162F00E4F58CF58AD2A9C28C22E2
:0B162400758DB1758BE0D2ABD28E2229
:03001B00020CC311
:100CC300C0E0C0F0C083C082C0D075D000C000C0F7
:100CD30001C002C003C004C005C006C007C28E75B0
:100CE3008DB1758BE0D28E78AAE61846600708E6C8
:100CF300161870011678ABE6600316800F78A4E629
:100D0300FF700974A52FF8E6FF1215E2D007D0068D
:100D1300D005D004D003D002D001D000D0D0D082EF
:070D2300D083D0F0D0E032D4
:100A2E004D55544500204C2B3000522B30200018D1
:100A3E00C608407806784268C070C270C618407802
:100A4E00C678C200006000008402940AD408400AEE
:100A5E005078C43A5210861A527086708430C66826
:100A6E00C41212084644A400860DC409E418C678C0
:100A7E008418E678A470C2121008C6048C0AD60533
:100A8E00280510140A621042414C414E4345440061
:100A9E0043440054554E455200415558310041557E
:100AAE0058320043494E454D41005441504500FFD8
:100ABE000A95FF0A9EFF0AA1FF0AA7FF0AACFF0ACA
:040ACE00B1FF0AB8B2
:100E36000E562020202020202020202020200000C8
:070E46000344000056C11F28
:1014D300E4FEC2A3EF30E004D2A58002C2A5D2A3EA
:0A14E300EFC313FF0EBE08EAD2A506
:0114ED0022DC
:10152000E4FFFEEFC313FFC2A300D2A330A5034321
:0615300007800EBE08ED6D
:011536002292
:10143D008F27C2A47F017E0012149BAF271214D3F5
:10144D007F017E0012149BD2A47F017E0002149BAB
:05141B002430FD7F0CF0
:10142000EFC394014016EFD3940D5010AB44AA457E
:0D143000A9461F8F82758300ED1209C422AA
:100EB7008B278A288929EFC39401404EEDD3940DDF
:100EC7005048EF9D50441F1DEFD39D503DAB27AABF
:100ED70028A92912094B601D0529E5297002052853
:100EE70014F912094BAB44AA45A946AC070F8C82EB
:100EF7007583008010AB44AA45A946AE070F8E82C2
:0B0F070075830074201209C480BE2214
:02139E00AE0798
:1013A000EE75F00A84FC60052430FD80027D207F0C
:1013B0000B121420EE75F00A84ACF0EC12141B7DB5
:0B13C000207F0A1214207F0D02142071
:1014B700301D0D7BFF7A0A792E7D0D7F0A020EB74C
:0C14C7007899E6249CF8E6FF12139E22A0
:100846008F267D5D7F071214207BFF7A0A79337D20
:10085600047F01120EB77BFF7A0A79387D0D7F0A75
:10086600120EB7E526D39406406974FA2526F526B6
:1008760012141BE526D39403403574FD2526F52670
:100886007D5D7F08121420E526B401077D5B7F0994
:10089600121420E526B402077D5C7F09121420E5B8
:1008A600266403600302094A7D5D7F09020947E564
:1008B60026B401077D5B7F08121420E526B40207E3
:1008C6007D5C7F08121420E526640370777D5D7FCA
:1008D60008806EE526C39406506AC374069526F50D
:1008E600262430FD7F04121420E526D394034030DD
:1008F60074FD2526F5267D5D7F06121420E526B4B7
:1009060001060D7F05121420E526B402077D5F7FE0
:1009160005121420E5266403702A7D5D7F0580217B
:10092600E526B401077D5E7F06121420E526B40293
:10093600077D5F7F06121420E526B403077D5D7FE1
:0509460006121420223E
:10153700E4FFAB44AA45A9468F8275830074201245
:0615470009C40FBF0DEC0A
:01154D00227B
:1015E200AB44AA45A94690000DEF1209C4C21F22BE
:0C16020075440075450075464802153718
:1015F20075440075450075465678ABA607D21F2282
:03001E00C21F22DC
:1015C10078A4E6700B78A6E6FF1215E278AB76C830
:0115D10022F7
:10100D00E4FF301F2578ABE67003C21F22E4FE74A7
:10101D00642EF974482EF8E6FD67600874642EF8A6
:10102D00A6057F010EBE0DE7801BE4FE74642EF94C
:10103D0074562EF8E6FD67600874642EF8A6057FD9
:05104D00010EBE0EE7DC
:01105200227B
:060382008B278A2889295F
:10038800E4F52DAB27AA28A929852D8275830012AB
:1003980009641209E603BC0003CD20043D2B03DDEC
:1003A8002D03ED5B03FD5C040D5D041D5E042D5FF4
:1003B80000000450AB27AA28A929852D827583003F
:1003C800740A1209C4AB27AA28A929852D82758326
:1003D80000740A806EAB27AA28A929852D82758307
:1003E80000740B805EAB27AA28A929852D82758306
:1003F80000740C804EAB27AA28A929852D82758305
:1004080000740D803EAB27AA28A929852D82758303
:1004180000740E802EAB27AA28A929852D82758302
:1004280000740F801EAB27AA28A929852D82758301
:10043800007410800EAB27AA28A929852D82758300
:1004480000742B1209C48011AB27AA28A929852D6D
:100458008275830074D0120991AB27AA28A929852F
:100468002D8275830012096425E0243DF582E43469
:100478000AF583E4740193FFAB2AAA2BA92C75F023
:1004880003E52DA4F58285F083EF1209C4AB27AAF2
:1004980028A929852D8275830012096425E0243D49
:1004A800F582E4340AF583E493FFAB2AAA2BA92C3E
:1004B80075F003E52DA42401F582E435F0F583EF0A
:1004C8001209C4AB2AAA2BA92C75F003E52DA42484
:1004D80002F582E435F0F583E41209C4052DE52D13
:0704E800640D600302038BA9
:0104EF0022EA
:1010530012100DEF603E752A00752B00752C727B04
:10106300007A00796412038212100D7F4012143D3E
:10107300C2A47FC01214D3E4FD74722DF8E6FF12EC
:1010830014D30DBD27F3D2A47F0C12143D7871E65F
:04109300FF12143DF7
:011097002236
:100D2A004552522E0A0D00256263000A0D00002466
:100D3A000146024703350436051F062A07210828FB
:100D4A0009311033110E120B131E143E150116022F
:100D5A001703180F190420052106223D23382425DC
:100D6A002520260D272C285529563057315832125E
:100D7A0033133414351536163719381D3951405284
:060D8A0041534254431ADC
:090E4D00013A00013B00013900EB
:10156400758740759850E4F5BD75BE9075BF0175DB
:05157400BD03D2AC2212
:080003008F993099FDC299228A
:100C5800E53914602214603624FE604C2404705771
:100C6800E53B7056EF64336002802F753B017539A0
:100C7800018F3C753A0122EFC394304006EFD394BC
:100C880034400280158F3D753902753A0222EFC350
:100C980094304006EFD394394005753BFE80188F99
:100CA8003E753A0375390422EF640D6005753BFE05
:0A0CB8008003753B028000E4F5396B
:010CC200220F
:0300230002154E75
:07154E00C0E0C0D075D01011
:0A155500309807AF99C298120C58A5
:05155F00D0D0D0E03205
:10136F00C3EF648094B0400ED3EF648094B95006FD
:10137F0074D02FFF8018C3EF648094C1400ED3EF59
:0F138F00648094C6500674C92FFF80027FFF222E
:100FBE00900001120964FF12136FAE07EEC454F0D5
:100FCE00FE900002120964FF12136FEF4206ED64E9
:100FDE00037026FDED25E02438F582E4340DF5830B
:100FEE00E493B50610ED25E02439F582E4340DF5D1
:0E0FFE0083E493FF220DBD2CDB753BFE7FFFCD
:01100C0022C1
:100BE600E53B24FE6011240470677BFF7A0D792AA9
:100BF600120088E4F53B227BFF7A0D7931752831A6
:100C0600120088E4F524AD24ED3395E0FCC3ED95A0
:100C16003A7480F86C9850157BFF7A0D7931743CE4
:100C26002524F8E6F528120088052480D97BFF7A6A
:100C36000D7935120088E4F53BFB7A00793CAD3A34
:100C4600120FBEEFFD3395E0FCEDF44C6003120489
:010C5600F0AD
:010C5700227A
:1013F5001214EE12156412163912162F1216241233
:10140500000E120016120E57120BE6120D90301E2A
:06141500F712105380F2F3
:100AE4000213F5E493A3F8E493A34003F68001F220
:100AF40008DFF48029E493A3F85407240CC8C33313
:100B0400C4540F4420C8834004F456800146F6DFE1
:100B1400E4800B0102040810204080900DF5E47E6F
:100B2400019360BCA3FF543F30E509541FFEE493D6
:100B3400A360010ECF54C025E060A840B8E493A39D
:100B4400FAE493A3F8E493A3C8C582C8CAC583CAC8
:100B5400F0A3C8C582C8CAC583CADFE9DEE780BE80
:010E5600009B
:10094B00BB010689828A83E0225002E722BBFE02AA
:09095B00E32289828A83E49322DD
:10096400BB010CE58229F582E5833AF583E0225048
:1009740006E92582F8E622BBFE06E92582F8E22292
:0D098400E58229F582E5833AF583E49322AC
:10099100BB010FF8E58229F582E5833AF583E0286A
:1009A100F0225009C58229F8E58226F622BBFE090C
:1009B100C58229F8E22582F222F8EA2583F583E946
:0309C10093282256
:1009C400F8BB010DE58229F582E5833AF583E8F069
:1009D400225006E92582C8F622BBFE05E92582C815
:0209E400F222FD
:1009E600D083D082F8E4937012740193700DA3A3A0
:1009F60093F8740193F5828883E4737402936860B4
:060A0600EFA3A3A380DFB3
:10002600E5342428F8E605342278253017027828A6
:10003600E475F001120A1E02094B2010EB7F2ED246
:10004600108018EF540F2490D43440D4FF30140B92
:10005600EF24BFB41A0050032461FFE53560021592
:10006600350538E5387002053730170D7825E47503
:10007600F001120A1EEF020A0C0200037403D217E3
:100086008003E4C217F5348B258A268927E4F535E3
:10009600F537F538E53560077F2012006180F57584
:1000A60036FFC211C210C212C213C215C216C2183E
:1000B60012002FFF700D3017057F00120072AF3847
:1000C600AE3722B4255FC2D5C21412002FFF24D04A
:1000D600B40A00501A75F00A783530D50508B6FF0F
:1000E6000106C6A426F620D5047002D21380D924B0
:1000F600CFB41A00EF5004C2E5D214020272D21134
:1001060080C6D21080C0D21280BCD2D580BAD21599
:1001160080B47F201200612012077401B5350040BB
:10012600F1120026FF12006102009AD218D2168040
:1001360095120026FB120026FA120026F94A4B7089
:100146000679437A037BFF20122EE535602A7E006E
:100156008E8275830012096460060EEE653670F0B5
:10016600C2D5EBC0E0EAC0E0E9C0E0EE1202B9D0C9
:10017600E0F9D0E0FAD0E0FB12094BFF60AAEBC031
:10018600E0EAC0E0E9C0E0120061D0E02401F9D065
:10019600E03400FAD0E0FBE5360460DCD536D980E1
:1001A600877BFF7A0279B5D212809C79108002791A
:1001B60008C216C2188008D2D5790A8004790AC204
:1001C600D5E536047002F536E4FAFDFEFF12002688
:1001D600FC7B08201113120026FD7B1030100A123A
:1001E6000026FE120026FF7B20EC3382D592D550E6
:1001F60013C3E43010069FFFE49EFEE42011039D26
:10020600FDE49CFCE4CBF8C211EC700CCFCECDCC57
:10021600E824F8F870F38017C3EF33FFEE33FEEDF2
:1002260033FDEC33FCEB33FB994002FB0FD8E9EBD3
:10023600301105F8D0E0C448B211C0E00AEC4D4ECA
:100246004F78207B0070C2EAB5360040BCC0E01291
:1002560002BBD0F0D0E0201104C4C0E0C4B211C08B
:10026600F012004AD0F0D5F0EB02009A1209E6012E
:10027600375301B15801084C01044201B54F01BD85
:0F0286004401BD49011D4301C35501A74601A70E
:100295004501A747036350010C2D01102E01332B97
:1002A500011423013120034C2A00CC480000012B06
:1002B5003F3F3F00790AA2D5201314301509B91024
:1002C500020404B9080104A2D52016025001042035
:1002D50012689212B535005034C0E07F20301319F2
:1002E5007F30A21272167215500F120312C212C27B
:1002F50016C215C2187F30800F301503E9C0E01211
:100305000061301503D0E0F9D0E0B535CC301517D4
:100315007F30B9100C1200617F583014077F788048
:1003250003B908031200613012057F2D0200617FB9
:10033500202018F87F2B2016F322921280CF286EEA
:10034500756C6C2900D2111200263011F8C2117893
:100355003530D50108F60200CC2D5043495812001E
:10036500262403B405004001E490035E9312005275
:0D037500743A120052D2137535040201B122
:100A0C00BB010689828A83F0225002F722BBFE01C9
:020A1C00F322C3
:100A1E00FAE6FB0808E6F925F0F618E6CA3AF622D9
:00000001FF
